:020000020000FC
:100000000C94AB000C94C8000C94C8000C94C8006D
:100010000C94C8000C948E020C94C8000C94C80078
:100020000C94C8000C945D020C94C8000C94C80099
:100030000C94C8000C94C8000C94C8000C94C80020
:100040000C94C8000C94C8000C94C8000C94C80010
:100050000C94C8006E616E00696E660000407A10F4
:10006000F35A00A0724E18090010A5D4E80000E869
:100070007648170000E40B54020000CA9A3B0000C7
:1000800000E1F505000080969800000040420F0056
:100090000000A08601000000102700000000E80317
:1000A000000000006400000000000A0000000000E2
:1000B0000100000000002C76D888DC674F0823DFA1
:1000C000C1DFAE59E1B1B796E5E3E453C63AE65174
:1000D000997696E8E6C28426EB898C9B62ED407C9B
:1000E0006FFCEFBC9C9F40F2BAA56FA5F490055A37
:1000F0002AF75C936B6CF9676DC11BFCE0E40D475C
:10010000FEF520E6B500D0ED902E0300943577057E
:100110000080841E080000204E0A000000C80C3336
:100120003333330F986E12831141EF8D2114893BC5
:10013000E65516CFFEE6DB18D1844B381BF77C1D45
:10014000901DA4BBE424203284725E228100C9F198
:1001500024ECA1E53D2711241FBECFE5D8E0DEBF8A
:10016000CDBF10E0A0E6B0E0E0E6F1E102C005900E
:100170000D92A236B107D9F710E0A2E6B0E001C0B7
:100180001D92AF39B107E1F70E94AC020C94AF08A1
:100190000C9400000C94003E08958150E6E8F0E0D5
:1001A000E80FF11D80818BBBAC9A85818BBBAB9A2C
:1001B00082858BBBAA9A87858BBBA99A84898BBBC6
:1001C000A89A0895CF93DF93F894809165008823CF
:1001D00009F4A9C0E6E8F0E0DF0110821182128282
:1001E00013821482359650E0EF39F507B1F780910C
:1001F0006200909163002AE130E0829FF001839FCA
:10020000F00D929FF00D1124E050FC4EF093690028
:10021000E093680020916A0030916B0080916C003F
:10022000813009F409C184918093860031968491CC
:1002300080938B00319684918093900031968491C5
:10024000809395003196849180939A00759684915D
:1002500090E024E135E0A901849F9001859F300D55
:10026000949F300D11243BBD2ABD749784918093D7
:1002700087003196849180938C003196849180938D
:100280009100319684918093960031968491809369
:100290009B003BBD2ABD31968491809388003196A6
:1002A000849180938D003196849180939200319651
:1002B0008491809397003196849180939C003BBDFC
:1002C0002ABD3196849180938900319684918093E0
:1002D0008E0031968491809393003196849180931F
:1002E00098003196849180939D003BBD2ABD319644
:1002F000849180938A003196849180938F00319607
:1003000084918093940031968491809399003196E2
:10031000849180939E003BBD2ABD30936B00209357
:100320006A001092650012BA15BA1BBA979A8091AA
:100330006000813099F080916000823029F18091D5
:1003400060008330B9F180916000843009F45EC0B0
:1003500080916000853009F087C042C0809186009E
:100360008BBBAC9A80918B008BBBAB9A8091900039
:100370008BBBAA9A809195008BBBA99A80919A0019
:100380008BBBA89A929A70C0809187008BBBAC9A65
:1003900080918C008BBBAB9A809191008BBBAA9A09
:1003A000809196008BBBA99A80919B008BBBA89AE9
:1003B000939A5AC0809188008BBBAC9A80918D0033
:1003C0008BBBAB9A809192008BBBAA9A80919700CD
:1003D0008BBBA99A80919C008BBBA89A949A44C02D
:1003E00080918A008BBBAC9A80918F008BBBAB9ABB
:1003F000809194008BBBAA9A809199008BBBA99A9B
:1004000080919E008BBBA89A969A2EC080918900FD
:100410008BBBAC9A80918E008BBBAB9A8091930082
:100420008BBBAA9A809198008BBBA99A80919D0062
:100430008BBBA89A959A18C0EDE6F0E080818C936A
:100440008181ED018D8382818A8783818F87848179
:100450008C8B88B394E0892788BB3596119640E051
:10046000E638F40759F759CF9798109264007894BA
:10047000DF91CF910895CF93DF93CDE6D0E05F9BDE
:10048000FECF8CB189930E94E20080E0C638D80785
:10049000B1F75F9BFECF8CB18E3729F05D9BFECF0D
:1004A00085E48CB907C05D9BFECF8EE78CB981E0F7
:1004B00080936500DF91CF9108951F920F920FB640
:1004C0000F9211242F933F938F939F93F8948091D1
:1004D000660090916700209162003091630001975F
:1004E0008217930751F0809162009091630001960A
:1004F000909363008093620004C010926300109296
:10050000620081E08093650078949F918F913F9184
:100510002F910F900FBE0F901F9018951F920F9262
:100520000FB60F9211248F93F8948091600085305C
:1005300031F0809160008F5F8093600003C081E0A4
:100540008093600081E08093640078948F910F9095
:100550000FBE0F901F9018950F931F93CF93DF93AB
:100560000E9446039FEF9ABB84E087BB94BB91BB7C
:10057000C29A1BBA15BA12BA8EB588618EBD8FB5F4
:1005800083608FBD8EB583608EBD89B7846089BF5F
:1005900080E090E49BBD8ABD85B5836085BD85B54F
:1005A000886485BD8AE583BD89B7806489BFE0E83A
:1005B000F3E1E4918E2F90E09093670080936600C2
:1005C000E1E8F3E1E49120916600309167008E2F1D
:1005D00090E0982F8827820F931F90936700809355
:1005E000660078940DE610E080916400882301F5A0
:1005F0005F9BFACF8CB18A32F1F08332C9F18C342F
:10060000D9F581E080936C0089B78B7F89BFF801B1
:10061000119280E0E638F807D9F781E08093650011
:100620005D9BFECF8CE48CB980916400882301F33C
:100630000E94E200DDCFE8015F9BFECF8CB1899381
:100640000E94E20080E0C638D807B1F75F9BFECF7A
:100650008CB18E3729F05D9BFECF85E48CB9C4CF79
:100660005D9BFECF8EE78CB981E080936500BCCFA7
:1006700012BA0C94003EB8CF8E3409F0B5CF109268
:100680006C00C29A89B7846089BFAECF10BC8BE082
:1006900089B988E18AB986E880BD8CB15F99FDCFC0
:1006A0000895A0E1B0E0E7E5F3E00C9478084C0190
:1006B0003B017A01FC0117821682838181FD06C00D
:1006C0008FEF9FEF99C3EC84FD8405C09E012F5FDF
:1006D0003F4F388B2F87F4013381F30133FD859130
:1006E00033FF81913F01882309F483C3853239F4B4
:1006F00033FD859133FF81913F01853229F4B401A7
:1007000090E00E94EE07E7CF982FBB241E86AA2414
:10071000FFE1FB15C8F09B3269F09C3228F490325F
:1007200059F0933289F40DC09D3241F0903361F459
:1007300021E021C042E0B42A84E029C098E0B92A2F
:100740002AC0E0E1BE2A27C0B7FC2EC0292F2053C3
:100750002A3098F4B6FE07C08AE0A89EC001112492
:10076000A22EA80E18C08AE0FE85F89FC0011124B1
:10077000280F2E8720E2B22A0EC09E3229F4B6FC42
:1007800038C340E4B42A07C09C3619F480E8B82A7C
:1007900002C0983649F4F30133FD959133FF9191EE
:1007A0003F01992309F0B4CF892F8554833020F479
:1007B0008B2D8061905E07C0892F8556833008F0AD
:1007C000AFC18B2D8F7E86FD02C076E0A72E6FE332
:1007D000B62EB822953619F4F0E4BF2A07C0963633
:1007E00019F420E8B22A02C0A110AA94B7FE0AC0E8
:1007F0003BE33A1518F45CE3552E02C05A2C53948F
:1008000027E007C047E04A1510F447E0A42E2A2D40
:100810005524C70104969D878C87F70160817181FB
:1008200082819381052DAE014F5F5F4F0E940007CB
:100830006C010981202E332400FF04C003FD02C097
:100840001DE209C0B1FE02C01BE205C0B2FE02C03B
:1008500010E201C010E0C1018C709070892B09F486
:100860003DC0112311F084E001C083E0FE858F17A5
:1008700010F01E860FC02E85281B2E87B3FC0AC0E1
:10088000B40180E290E00E94EE073E8531503E8741
:100890003323B1F7112329F0B401812F90E00E9496
:1008A000EE0723FE03C004E510E00EC008E510E0EB
:1008B0000BC0E114F10409F08052B40190E00E94F1
:1008C000EE070F5F1F4F05C0EB2CFF2440E1E42231
:1008D000FF24F8018491882361F787C2B7FE12C014
:1008E0005C0C24FE04C08A81813309F45A941514E7
:1008F0001CF0552453942FC0F8E0F51560F538E04E
:10090000532E29C0B6FC27C08A2D90E08C159D057A
:100910004CF02CEFC2162FEFD20624F030E8B32AA9
:1009200001C0AA94AA2049F0E2E0F0E0EC0FFD1F1C
:10093000EA0DF11D80818033A1F3B7FE0CC08A2D32
:1009400090E0C816D90614F080E002C08A2D8C19F8
:100950005A2C5394A82EB7FC03C025E030E009C000
:100960001C141D041CF021E030E003C096012F5F31
:100970003F4F112311F02F5F3F4FAA2029F08A2DFE
:1009800090E00196280F391F4E85842F90E028179C
:10099000390714F01E8603C08E85821B8E87EB2CD0
:1009A000FF24C70189709070892B49F00BC0B401F6
:1009B00080E290E00E94EE079E8591509E87EE8532
:1009C000EE23A9F7112329F0B401812F90E00E94B2
:1009D000EE07E3FE09C00BC0B40180E390E00E9483
:1009E000EE07FE85F150FE872E852223A9F7B7FE7C
:1009F00048C08601D7FE02C000E010E076010894EE
:100A0000E11CF11CE01AF10A81E090E08C0F9D1FBF
:100A1000E80EF91EF601E519F1092F018A2D90E083
:100A2000AA24BB24A81AB90AFFEF0F3F1F0729F415
:100A3000B4018EE290E00E94EE07C016D10634F0B9
:100A4000401651061CF4F701808101C080E301507B
:100A500010400894E11CF11C0A151B052CF0B40190
:100A600090E00E94EE07E0CF0C151D0539F42A81B5
:100A7000263318F4253311F424FE81E3B40190E009
:100A80004CC08A81813309F00F7EB40190E00E944E
:100A9000EE07AA20A1F0B4018EE290E00E94EE07DA
:100AA00012E0E1E0F0E0EC0FFD1FE10FF11D8081AD
:100AB0001F5FB40190E00E94EE07AA9491F7E4FE54
:100AC00003C085E490E002C085E690E0B4010E9496
:100AD000EE07D7FC05C0C114D10441F404FF06C0E1
:100AE000D094C194D108D3948DE201C08BE2B401BB
:100AF00090E00E94EE0780E305C08F5F26EF3FEF96
:100B0000C20ED31E3AE0C316D104BCF7B40190E084
:100B10000E94EE07B401C601C0960E94EE0765C1AF
:100B2000933631F0933791F0933509F064C025C0C6
:100B3000C70102969D878C87F701808189838E018A
:100B40000F5F1F4F21E0C22ED12C13C0F70100818F
:100B50001181B6FC03C06FEF7FEF02C06A2D70E019
:100B600097012E5F3F4F3D872C87C8010E94E30706
:100B70006C019FE7F92EFB2016C0F701008111815F
:100B8000B6FC03C06FEF7FEF02C06A2D70E09701E3
:100B90002E5F3F4F3D872C87C8010E94D8076C010C
:100BA00080E8F82EFB28F3FE09C021C0B40180E2E2
:100BB00090E00E94EE073E8531503E874E85842F9F
:100BC00090E0C816D90690F312C0F801F7FC8591A1
:100BD000F7FE81918F01B40190E00E94EE07FE853F
:100BE000FF2311F0F150FE870894C108D108C11409
:100BF000D10459F7FAC0943611F0993691F5B7FE41
:100C00000BC097012C5F3F4F3D872C87F701608118
:100C10007181828193810EC097012E5F3F4F3D8786
:100C20002C87F701808191819C01B901882777FD8C
:100C30008095982F0B2D0F7697FF08C09095809583
:100C4000709561957F4F8F4F9F4F00682AE030E08D
:100C5000AE014F5F5F4F0E941A08D82E3F85D31A0E
:100C600044C0953729F41B2D1F7E2AE030E01DC0BB
:100C70001B2D197F9F3661F0903720F4983509F0CD
:100C8000B8C00FC0903739F0983709F0B2C004C02F
:100C900028E030E00AC0106114FD146020E130E06B
:100CA00004C014FD166020E132E017FF0AC0C7013E
:100CB00004969D878C87F701608171818281938181
:100CC0000AC0C70102969D878C87F70180819181B8
:100CD000BC0180E090E0AE014F5F5F4F0E941A08B8
:100CE000D82EFF85DF1A012F0F7706FF09C00E7F70
:100CF000DA1430F404FF06C002FD04C00F7E02C007
:100D00001D2D01C01A2D04FF0CC0FE01ED0DF11DBB
:100D10008081803311F4097E08C01F5F02FF05C087
:100D200003C0802F867809F01F5FE02E03FD16C0F8
:100D300000FF10C02E85121710F0AD2C0BC0AE8432
:100D4000AD0CA11A1E8506C0B40180E290E00E949D
:100D5000EE071F5F3E851317B8F306C04E851417C4
:100D600018F4411B4E8701C01E86E4FE10C0B4017A
:100D700080E390E00E94EE07E2FE1EC0E1FE03C0A9
:100D800088E590E002C088E790E0B4010CC08E2DA9
:100D9000867891F0E1FE02C08BE201C080E207FD9F
:100DA0008DE2B40190E00E94EE0706C0B40180E33A
:100DB00090E00E94EE07AA94DA14C0F3DA94E1E01E
:100DC000F0E0EC0FFD1FED0DF11D8081B40190E00E
:100DD0000E94EE07DD2049F0F1CFB40180E290E0FF
:100DE0000E94EE078E8581508E879E859923A9F7F4
:100DF0006ACCF40186819781E2E160960C949408B4
:100E0000283008F027E03327DA01990F311D87FDDC
:100E1000916000966105710539F432602E5F3D9353
:100E200030E32A95E1F708959F3F30F0803871054F
:100E3000610509F03C5F3C5F3D93913008F08068AC
:100E4000911DDF93CF931F930F93FF92EF92192F72
:100E5000987F9695E92F96959695E90FFF27EA5486
:100E6000FF4F99273327EE24FF24A701E7010590C0
:100E70000894079428F4360FE71EF81E491F511DE9
:100E8000660F771F881F991F0694A1F70590079496
:100E900028F4E70EF81E491F561FC11D770F881F43
:100EA000991F661F0694A1F70590079428F4F80E81
:100EB000491F561FC71FD11D880F991F661F771F17
:100EC0000694A1F70590079420F4490F561FC71FF9
:100ED000D81F990F661F771F881F0694A9F7849162
:100EE0001095177041F0D695C79557954795F7948B
:100EF000E7941A95C1F7ECE5F0E068941590159128
:100F000035916591959105907FE27395E118F10A0D
:100F1000430B560BC90BD009C0F7E10CF11E431F60
:100F2000561FC91FD01D7EF4703311F48A95E6CF89
:100F3000E894015030F0080F0AF40027021708F473
:100F4000202F2395022F7A3328F079E37D932A9579
:100F5000E9F710C07D932A9589F6069497956795D1
:100F6000379517951794E118F10A430B560BC90BE7
:100F7000D00998F023957E9173957A3308F070E349
:100F80007C932013B8F77E9170617D9330F0839548
:100F900071E37D9370E32A95E1F71124EF90FF90C0
:100FA0000F911F91CF91DF91992787FD909508951B
:100FB000FC010590615070400110D8F78095909524
:100FC0008E0F9F1F0895FC01615070400190011029
:100FD000D8F7809590958E0F9F1F08950F931F93BC
:100FE000CF93DF938C01EB018B8181FF1BC082FFCC
:100FF0000DC02E813F818C819D812817390764F4B3
:10100000E881F9810193F983E88306C0E885F985D1
:10101000802F0995892B31F48E819F8101969F83C2
:101020008E8302C00FEF1FEFC801DF91CF911F9198
:101030000F910895FA01AA27283051F1203181F14A
:10104000E8946F936E7F6E5F7F4F8F4F9F4FAF4FD0
:10105000B1E03ED0B4E03CD0670F781F891F9A1FE3
:10106000A11D680F791F8A1F911DA11D6A0F711D97
:10107000811D911DA11D20D009F468943F912AE0A3
:10108000269F11243019305D3193DEF6CF0108958B
:10109000462F4770405D4193B3E00FD0C9F7F6CFBC
:1010A000462F4F70405D4A3318F0495D31FD405284
:1010B000419302D0A9F7EACFB4E0A695979587951A
:1010C00077956795BA95C9F70097610571050895F9
:1010D0009B01AC010A2E06945795479537952795A5
:1010E000BA95C9F7620F731F841F951FA01D08953D
:1010F0002F923F924F925F926F927F928F929F9228
:10110000AF92BF92CF92DF92EF92FF920F931F9315
:10111000CF93DF93CDB7DEB7CA1BDB0B0FB6F894C6
:10112000DEBF0FBECDBF09942A88398848885F8406
:101130006E847D848C849B84AA84B984C884DF8077
:10114000EE80FD800C811B81AA81B981CE0FD11D5B
:101150000FB6F894DEBF0FBECDBFED010895FFCFEF
:101160000100FFFFFFFFFFFFFFFFFFFFFFFFFFFF8C
:10117000FFFFFFFFFFFFFFFFFFFFFFFFFFFFFFFF7F
:10118000FFFFFFFFFFFFFFFFFFFFFFFFFFFFFFFF6F
:10119000FFFFFFFFFFFFFFFFFFFFFFFFFFFFFFFF5F
:1011A000FFFFFFFFFFFFFFFFFFFFFFFFFFFFFFFF4F
:101380002701FFFFFFFFFFFFFFFFFFFFFFFFFFFF43
:10139000FFFFFFFFFFFFFFFFFFFFFFFFFFFFFFFF5D
:1013A000FFFFFFFFFFFFFFFFFFFFFFFFFFFFFFFF4D
:1013B000FFFFFFFFFFFFFFFFFFFFFFFFFFFFFFFF3D
:1013C000FFFFFFFFFFFFFFFFFFFFFFFFFFFFFFFF2D
:1013D000FFFFFFFFFFFFFFFFFFFFFFFFFFFFFFFF1D
:1013E000FFFFFFFFFFFFFFFFFFFFFFFFFFFFFFFF0D
:1013F000FFFFFFFFFFFFFFFFFFFFFFFFFFFFFFFFFD
:1014000000000000000000000000000000000000DC
:101410000000000000000000000A000000000000C2
:1014200000000000000000000000000000000000BC
:101430000000000A000000000000000000000000A2
:10144000000000000000000011000000110A000070
:10145000000000000000000000000000000000008C
:1014600000001B1100111B0A00000000000000001A
:101470000000000000000000000000001F1111111A
:101480001F0A000000000000000000000000000033
:101490000011000000111F1111111F0A00000000AF
:1014A00000000000000011000000111100000011F8
:1014B0001F1111111F0A000000000011000000118F
:1014C000110000001111000000111F1111111F0A5D
:1014D0001100000011110000001111000000111195
:1014E000000000111F1111111F0A1B11001113110F
:1014F00000000011110000001111000000111F1167
:1015000011111F0A1F1111111F11000000111100EC
:1015100000001111000000111F1111111F0A1F1BE3
:10152000111B1F110000001111000000111100001B
:1015300000111F1111111F0A1F1F1B1F1F11000077
:101540000011110000001111000000111F111111F4
:101550001F0A1F1F1F1F1F11000000111100000094
:101560001111000000111F1111111F0A00000000CD
:10157000001F1F1F1F1F110000001111000000118C
:101580001F1111111F0A00000000000000000000E0
:101590001F1F1F1F1F11000000111F1111111F0A13
:1015A0000000000000000000000000000000001F1C
:1015B0001F1F1F1F1F1111111F0A00000000000034
:1015C00000000000000000000000000000001F1FDD
:1015D0001F1F1F0A000000000000000000000000A4
:1015E000000000000000000000000000000A0000F1
:1015F00000000000000000000000000000000000EB
:10160000000000000000000A0000100000000010B0
:10161000000010101010100000100000000010005A
:10162000000A000008000000000800000808080880
:1016300008000008000000000800000A0000040084
:10164000000000040000040404040400000400007E
:1016500000000400000A0000040000000004000074
:101660000102040810000004000000000400000A49
:101670000000040000000004000000001F00000043
:101680000004000000000400000A00000400000044
:101690000004000010080402010000040000000023
:1016A0000400000A0000040000000004000004041C
:1016B000040404000004000000000400000A00000C
:1016C00004000000000400000102040810000004EF
:1016D000000000000400000A0000040000000004F4
:1016E000000000001F0000000004000000000400D3
:1016F000000A0000040000000004000010080402BA
:1017000001000004000000000400000A00000400C2
:1017100000000004000004040404040000040000AD
:1017200000000400000A040000000400040004009B
:101730000000040000000400040004000000040A8B
:10174000000004000000000400000404040404007D
:101750000004000000000400000A0404040404045F
:101760000404040404040404040404040404040439
:101770000404040A01020408100102040810010212
:10178000040810010204081001020408100A0000F5
:101790001F000000001F000000001F000000001FCD
:1017A000000000001F00000A1008040201100804D5
:1017B00002011008040201100804020110080402CA
:1017C000010A0404040404040404040404040404D6
:1017D00004040404040404040404040A01020408C4
:1017E000100102040810010204081001020408108C
:1017F00001020408100A00001F000000001F000082
:1018000000001F000000001F000000001F00000A71
:10181000100804020110080402011008040201105B
:101820000804020110080402010A04040404040468
:101830000404040404040404040404040404040468
:101840000404040A10101010100808080808040402
:10185000040404020202020201010101010A000063
:1018600000000000000000001F1F1F1F1F000000DD
:10187000000000000000000A010101010102020253
:1018800002020404040404080808080810101010D8
:10189000100A0404040404040404040404040404F6
:1018A00004040404040404040404040A10101010C2
:1018B00010080808080804040404040202020202D2
:1018C00001010101010A0000000000000000000009
:1018D0001F1F1F1F1F000000000000000000000A63
:1018E00001010101010202020202040404040408CD
:1018F0000808080810101010100A04040404040456
:101900000404040404040404040404040404040497
:101910000404040A02020202020202020202020299
:10192000020202020202020202020202020A010191
:101930000101010101010101010101010101010197
:10194000010101010101010A00000101070000017C
:10195000010700000101070000010107000001016B
:10196000070A000000001F000000001F0000000028
:101970001F000000001F000000001F0A00001010E0
:101980001C000010101C000010101C000010101C87
:10199000000010101C0A1010101010101010101061
:1019A0001010101010101010101010101010100A3D
:1019B0001C101000001C101000001C101000001C57
:1019C000101000001C101000000A1F000000001F73
:1019D000000000001F000000001F000000001F00AA
:1019E0000000000A070101000007010100000701D3
:1019F000010000070101000007010100000A0101C8
:101A000001010101010101010101010101010101C6
:101A1000010101010101010A0000000000000000B5
:101A200000000000000000000000000000000000B6
:101A3000000A00000000000000000000000000009C
:101A40000000000000001F1F1F1F1F0500000000F6
:101A500000000000000000000000001F1111111F15
:101A6000000E0A0E0005000000000000000000004B
:101A70001F1111111F000E0A0E00000004000005C6
:101A800000000000001F1111111F000E0A0E0000BF
:101A9000000400000000000000051F1111111F00CC
:101AA0000E0A0E000000040000000000000000000C
:101AB000000000051F1F1B1F1F0000040000000086
:101AC00000000000000000000000000000051F1FD3
:101AD0001F1F1F00000000000000000000000000A9
:101AE0000000000000000005000E0A0E001F11118A
:101AF000111F0000000000000000000000000000B6
:101B000000050000040000000E0A0E001F11111154
:101B10001F000000000000000000000500000000A1
:101B2000000000040000000E0A0E001F1111111F1A
:101B300000000000000500000000000000000000A0
:101B40000000040000000E0A0E001F1111111F05F5
:101B50000000000000000000000000000000000085
:101B6000000400001F1F1B1F1F05000000000000D5
:101B700000000000000000000000000000001F1F27
:101B80001F1F1F05000000000000000000000000F3
:101B90000000001F1111111F000E0A0E00050000A9
:101BA00000000000000000001F1111111F000E0AAC
:101BB0000E0000000400000500000000001F1111CD
:101BC000111F000E0A0E00000004000000000000BB
:101BD00000051F1111111F000E0A0E000000040065
:101BE0000000000000000000000000051F1F1B1F78
:101BF0001F000004000000000000000000000000C2
:101C00000000000000051F1F1F1F1F000000000034
:101C100000000000000000000000000000000005BF
:101C2000000E0A0E001F1111111F0000000000001D
:101C3000000000000000000000050000040000009B
:101C40000E0A0E001F1111111F00000000000000FD
:101C50000000000500000000000000040000000E6D
:101C60000A0E001F1111111F0000000000050000E6
:101C700000000000000000000000040000000E0A48
:101C80000E001F1111111F050000000000000000D0
:101C90000000000000000000000400001F1F1B1FC8
:101CA0001F05000000000000000000000000000010
:101CB0000000000000001F1F1F1F1F050000000084
:101CC00000000000000000000000001F1111111FA3
:101CD000000E0A0E000500000000000000000000D9
:101CE0001F1111111F000E0A0E0000000400000554
:101CF00000000000001F1111111F000E0A0E00004D
:101D0000000400000000000000051F1111111F0059
:101D10000E0A0E0000000400000000000000000099
:101D2000000000051F1F1B1F1F0000040000000013
:101D300000000000000000000000000000051F1F60
:101D40001F1F1F0000000000000000000000000036
:101D50000000000000000005000E0A0E001F111117
:101D6000111F000000000000000000000000000043
:101D700000050000040000000E0A0E001F111111E2
:101D80001F0000000000000000000005000000002F
:101D9000000000040000000E0A0E001F1111111FA8
:101DA000000000000005000000000000000000002E
:101DB0000000040000000E0A0E001F1111111F0583
:101DC0000000000000000000000000000000000013
:101DD000000400001F1F1B1F1F0500100010001033
:101DE0001010101010101010100010101000000033
:101DF0001000000A00080008000808080808080881
:101E0000080808000808080000000800000A00048C
:101E1000000400040404040404040404040004048E
:101E2000040000000400000A00080002001008047A
:101E3000020110080402010008040200000004006E
:101E4000000A00000A000000001F000000001F0040
:101E50000000000E000000000400000A000200085C
:101E60000001020408100102040810000204080026
:101E700000000400000A0004000400040404040438
:101E80000404040404000404040000000400000A24
:101E900000080002001008040201100804020100FA
:101EA0000804020000000400000A00000A0000000C
:101EB000001F000000001F000000000E00000000D6
:101EC0000400000A000200080001020408100102D8
:101ED000040810000204080000000400000A0004C6
:101EE00000040004040404040404040404000404BE
:101EF000040000000400000A0004000400040E0EA8
:101F00000E04040E0E0E0400040E04000000040073
:101F1000000A00040004000404040404040404048B
:101F200004000404040000000400000A000400048B
:101F300000040E0E0E04040E0E0E0400040E040027
:101F400000000400000A0008000200100E0E0E013E
:101F5000100E0E0E01000A040A0000000400000A20
:101F600000000A0000000E1F0E00000E1F0E0000F1
:101F7000040E040000000400000A00020008000132
:101F80000E0E0E10010E0E0E10000A040A000000C4
:101F90000400000A0004000400040E0E0E04040EE7
:101FA0000E0E0400040E040000000400000A0000ED
:101FB0000000000000000000000000000000000021
:101FC000000000000000000A000000000000000007
:101FD0000000000000000000000000000000000001
:101FE000000A01020408100102040810010204089A
:101FF00010010204081001020408101400001F0060
:102000000000001F000000001F000000001F000073
:1020100000001F000014100804020110080402014F
:10202000100804020110080402011008040201143F
:102030000404040404040404040404040404040460
:102040000404040404040404040F0102040810013D
:102050000204081001020408100102040810010221
:102060000408100F00001F000000001F0000000007
:102070001F000000001F000000001F00000F1008DC
:1020800004020110080402011008040201100804EF
:10209000020110080402010F0404040404040404EF
:1020A00004040404040404040404040404040404F0
:1020B000040A0102040810010204081001020408C5
:1020C00010010204081001020408100A00001F0099
:1020D0000000001F000000001F000000001F0000A3
:1020E00000001F00000A1008040201100804020189
:1020F0001008040201100804020110080402010A79
:10210000040404040404040404040404040404048F
:102110000404040404040404040501020408100176
:102120000204081001020408100102040810010250
:102130000408100500001F000000001F0000000040
:102140001F000000001F000000001F000005100815
:10215000040201100804020110080402011008041E
:102160000201100804020105040404040404040428
:10217000040404040404040404040404040404041F
:1021800004030102040810010204081001020408FB
:1021900010010204081001020408100300001F00CF
:1021A0000000001F000000001F000000001F0000D2
:1021B00000001F00000310080402011008040201BF
:1021C00010080402011008040201100804020103AF
:1021D00004040404040404040404040404040404BF
:1021E00004040404040404040402010204081001A9
:1021F0000204081001020408100102040810010280
:102200000408100200001F000000001F0000000072
:102210001F000000001F000000001F000002100847
:10222000040201100804020110080402011008044D
:10223000020110080402010204040404040404045A
:10224000040404040404040404040404040404044E
:102250000401000000000000000000000000000079
:1022600000000000000000000000000A0100000063
:102270001002000000080400000004080000000232
:1022800010101101010A00001100000001001000EF
:10229000010000001002000000081C000000070AF6
:1022A00010000000010010000100000011000000FB
:1022B00001001000070000001C0A040000000408D0
:1022C00000000002100000000100100001000101E8
:1022D0001110100A010000001002000000080400A4
:1022E000000004080000000210101101010A0000A3
:1022F00011000000010010000100000010020000A9
:1023000000081C000000070A100000000100100077
:102310000100000011000000010010000700000093
:102320001C0A040000000408000000021000000065
:1023300001001000010001011110100A010000004D
:102340001002000000080400000004080000000261
:1023500010101101010A000011000000010010001E
:10236000010000001002000000081C000000070A25
:10237000100000000100100001000000110000002A
:1023800001001000070000001C0A040000000408FF
:102390000000000210000000010010000100010117
:1023A0001110100A010000001002000000080400D3
:1023B000000004080000000210101101010A0000D2
:1023C00011000000010010000100000010020000D8
:1023D00000081C000000070A1000000001001000A7
:1023E00001000000110000000100100007000000C3
:1023F0001C0A040000000408000000021000000095
:1024000001001000010001011110100A010000007C
:102410001002000000080400000004080000000290
:1024200010101101010A000000000000000000006F
:102430000000000000000000000000000000000A92
:10244000000000000000000000000000000000008C
:102450000000030300000003030A00000000000066
:102460000000000000000000000000030300000066
:102470000303000A0000000000000000000000004C
:10248000000000000303000000030300000A000036
:102490000000000000000000000000000003030036
:1024A000000003030000000A00000000000000001C
:1024B0000000000000000006060000000606000004
:1024C000000A000000000000000000000000000002
:1024D000000C0C0000000C0C0000000A00000000C2
:1024E00000000000000000000000001818000000BC
:1024F00018180000000A00000000000000000000A2
:102500000000000000001818000000181800000A61
:1025100000000000000000000000000000000000BB
:102520000018180000001818000A00000000000041
:10253000000000000000000000000000181800006B
:102540000018180A00000000000000000000000051
:10255000001818000000181800000000000A000011
:10256000000000000000181800000018180000000B
:10257000000000000000000A000000181800000021
:10258000181800000000000000000000000000001B
:10259000000A0000000C0C0000000C0C0000000001
:1025A00000000000000000000000000A000000061B
:1025B0000600000006060000000000000000000009
:1025C00000000000000A00000606000000060600E9
:1025D0000000000000000000000000000000000AF1
:1025E00000060600000006060000000000000000D3
:1025F0000000000000000000000A060600000006BF
:1026000006000000000000000000000000000000C4
:102610000000000A030300000003030000000000A4
:10262000000000000000000000000000000A01019E
:102630000000000101000000000000000000000098
:10264000000000000000000A000000000000000080
:10265000000000000000000000000000000000007A
:10266000000A000000000000000000000000000060
:1026700000000000000000000000000A1F1F1F1FD4
:102680001F0000000000000000000000000000002B
:1026900000000000000A1F1F1F1F1700000000009D
:1026A0000000000000000000000000000000080A18
:1026B0001F1F1D1F17000000000000000000000089
:1026C0000000000000000200080A171F1D1F17006D
:1026D00000000000000000000000000000000800F2
:1026E0000200080A171F1D1B170000000000000051
:1026F000000000000000000008000204080A161F85
:102700001D1B17000000000000000000000000007A
:10271000000009000204080A161B1D1B1700000018
:102720000000000000000000000000000904020496
:10273000080A161B1D1B1600000000000000000008
:1027400000000000000009040204090A161B151B02
:102750001600000000000000000000000000000063
:1027600009040A04090A161B151B140000000000C6
:102770000000000000000000000009040A040B0A29
:10278000161A151B140000000000000000000000D5
:102790000000000009050A040B0A161A150B1400A4
:1027A000000000000000000000000000000009051B
:1027B0000A140B0A121A1509140000000000000088
:1027C00000000000000000000D050A160B0A021AA6
:1027D00015081400000000000000000000000000C8
:1027E00000001D050A170B0A02121508040000005C
:1027F0000000000000000000000000001D0D0A178E
:102800001B0A021001080400000000000000000084
:102810000000000000001D0F1E171B0A020001002F
:1028200004000000000000000000000000000000A4
:102830001D1F1E1F1B0A00000000000000000000FA
:10284000000000000000000000001F1F1F1F1F0AE3
:102850000000000000000000000000000000000078
:102860000000000000000000100500000000000053
:102870000000000000000000000000000000000058
:102880000010100A0000000000000000000000001E
:10289000000000000000000000001010100A0000FE
:1028A0000000000000000000000000000000000028
:1028B000000000101010100A0000000000000000CE
:1028C00000000000000000000000000010101010C8
:1028D000100A0000000000000000000000000000DE
:1028E00000000000000018101010100A0000000086
:1028F00000000000000000000000000000000000D8
:1029000018181010100A000000000000000000005D
:102910000000000000000000000018181810100A45
:1029200000000000000000000000000000000000A7
:102930000000000018181818100A0000000000001D
:102940000000000000000000000000000000181857
:102950001818180A00000000000000000000000025
:102960000000000000000000181818181C0A0000E1
:102970000000000000000000000000000000000057
:1029800000001818181C1C0A0000000000000000BD
:1029900000000000000000000000000018181C1CCF
:1029A0001C0A000000000000000000000000000001
:1029B000000000000000181C1C1C1C0A0000000085
:1029C0000000000000000000000000000000000007
:1029D0001C1C1C1C1C0A0000000000000000000061
:1029E000000000000000000000001E1C1C1C1C0A4F
:1029F00000000000000000000000000000000000D7
:102A0000000000001E1E1C1C1C0A0000000000002C
:102A100000000000000000000000000000001E1E7A
:102A20001E1C1C0A00000000000000000000000046
:102A300000000000000000001E1E1E1E1C0A0000F8
:102A40000000000000000000000000000000000086
:102A500000001E1E1E1E1E0A0000000000000000D6
:102A60000000000000000000000000001E1E1E1EEE
:102A70001F0A00000000000000000000000000002D
:102A80000000000000001E1E1E1F1F0A00000000A4
:102A90000000000000000000000000000000000036
:102AA0001E1E1F1F1F0A0000000000000000000083
:102AB000000000000000000000001E1F1F1F1F0A72
:102AC0000000000000000000000000000000000006
:102AD000000000001F1F1F1F1F0A00000000000051
:102AE00000000000000000000001000000001F1FA7
:102AF0001F1F1F0A0000000000000000000001006E
:102B000000000001000000001F1F1F1F1F0A00001F
:102B100000000001000000000100000000010000B2
:102B200000001F1F1F1F1F0A0100000000010000FE
:102B30000000010000000001000000001F1F1F1F17
:102B40001F0A010100000001000000000100000058
:102B50000001000000001F1F1F1F1F0A01010100CC
:102B60000001000000000100000000010000000062
:102B70001F1F1F1F1F0A01010101000100000000AB
:102B8000010000000001000000001F1F1F1F1F0A9E
:102B9000010101010101000000000100000000012D
:102BA000000000001F1F1F1F1F0A01010101030178
:102BB00000000000010000000001000000001F1FD5
:102BC0001F1F1F0A01010103030100000000010093
:102BD00000000001000000001F1F1F1F1F0A01014D
:102BE00003030301000000000100000000010000D9
:102BF00000001F1F1F1F1F0A010303030301000022
:102C00000000010000000001000000001F1F1F1F46
:102C10001F0A03030303030100000000010000007A
:102C20000001000000001F1F1F1F1F0A07030303EE
:102C3000030100000000010000000001000000008E
:102C40001F1F1F1F1F0A07070303030100000000C7
:102C5000010000000001000000001F1F1F1F1F0ACD
:102C60000707070303010000000001000000000146
:102C7000000000001F1F1F1F1F0A0707070703018F
:102C800000000000010000000001000000001F1F04
:102C90001F1F1F0A070707070701000000000100A8
:102CA00000000001000000001F1F1F1F1F0A070770
:102CB00007070F01000000000100000000010000F4
:102CC00000001F1F1F1F1F0A0707070F0F0100002B
:102CD0000000010000000001000000001F1F1F1F76
:102CE0001F0A07070F0F0F0100000000010000007E
:102CF0000001000000001F1F1F1F1F0A070F0F0FFA
:102D00000F010000000001000000000100000000B1
:102D10001F1F1F1F1F0A0F0F0F0F0F0100000000C2
:102D2000010000000001000000001F1F1F1F1F0AFC
:102D30001F0F0F0F0F010000000001000000000135
:102D4000000000001F1F1F1F1F0A1F1F0F0F0F0172
:102D500000000000010000000001000000001F1F33
:102D60001F1F1F0A1F1F1F0F0F010000000001007F
:102D700000000001000000001F1F1F1F1F0A1F1F6F
:102D80001F1F0F01000000000100000000010000F3
:102D900000001F1F1F1F1F0A1F1F1F1F1F010000F2
:102DA0000000010000000001000000001F1F1F1FA5
:102DB0001F0A1F1F1F1F1F0100000010010000003D
:102DC0000001000000001F1F1F1F1F0A1F1F1F1FE1
:102DD0001F010000001001000000100100000000B1
:102DE0001F1F1F1F1F0A1F1F1F1F1F010000001092
:102DF000010000001001000000101F1F1F1F1F0A0C
:102E000000000000000000000000000000000000C2
:102E10000000000000000000000A1F1F1F1F1F1FEE
:102E20001F1F1F1F1F1F1F1F1F1F1F1F1F1F1F1FB2
:102E30001F1F1F0A0000000000000000000000002B
:102E4000000000000000000000000000000A1F1F3A
:102E50001F1F1F1F1F1F1F1F1F1F1F1F1F1F1F1F82
:102E60001F1F1F1F1F1F1F0A00000000000000007F
:102E70000000000000000000000000000000000052
:102E8000000A000000000000000000000000000038
:102E900000000000000010000000000A0000000018
:102EA0000000000000000000000000000000000022
:102EB00018180000000A00000000000000000000D8
:102EC0000000000000181800000018180000000A98
:102ED0000000000000000000000000000000001CD6
:102EE0001C1C00001C1C1C00000A0000000000004C
:102EF000000000001E1E1E1E001C1C1C1E001E1EAC
:102F00001E1E000A00000000001F1F1F1F1F1F1FA2
:102F10001F1F1F1F1F1F1F1F1F1F1F1F1F0A1F1FD6
:102F20001F1F1F1F1F1F1F1F1F1F1F1F1F1F1F1FB1
:102F30001F1F1F1F1F1F1F0A0000000000000000AE
:102F40000000000000000000000000001000000071
:102F5000000A000000000000000000000000000067
:102F600000000000000018180000000A0000000027
:102F70000000000000000000000000181800000021
:102F800018180000000A0000000000000000000007
:102F900000000000001C1C1C00001C1C1C00000A7F
:102FA000000000000000000000001E1E1E1E001C8D
:102FB0001C1C1E001E1E1E1E000A00000000001F1A
:102FC0001F1F1F1F1F1F1F1F1F1F1F1F1F1F1F1F11
:102FD0001F1F1F0A1F1F1F1F1F1F1F1F1F1F1F1F16
:102FE0001F1F1F1F1F1F1F1F1F1F1F1F1F0A0F0530
:102FF000071E1D19150002061F0B17031E171711B8
:1030000005141A1C1A1A1E14171B050F0D191C1C67
:103010000F1C1D0E110B1414160E1A1E1B1D10165C
:103020000A141811040C1F05181C1F160307191B7E
:103030001F1005100E18081A1A030514030E060AAD
:10304000090D1004041E011B1B1507140519181186
:103050000F1E161E07140202100B13121210091174
:10306000171E13150C020E070F1F041F1C011B1443
:103070001D18110C011E1A08180B1115091D140A30
:103080000D15171D151B160D1D141416130C1416F3
:103090001A1C04010319091F170E0D080011171A35
:1030A0001D181F140E0C111B060A13040709051C1A
:1030B00003121D090E12161B141D07070314010A23
:1030C0001C1A140611001E031715021204090B1D09
:1030D000081C03090D1B051403061A1F0F0D1F1FE3
:1030E00000111619181813050D040B010B160C10FE
:1030F000041408080A1A1D01170E19190C121010D1
:103100001B070C1A1D030912060D0A1414130918C3
:103110001F09170200130A171E10100B0F11090DBB
:1031200002130C0B181401030C0A0300141E0E0BDF
:10313000081704060B08050015081711071F0314CC
:1031400009031A0E0817020109020B10160D050CCF
:103150000A171B130D0B0C060C14161B1E091A0B59
:103160000215021E111C16010F0A08080E15060E84
:1031700006130A150C0D190E1510101A0814101547
:1031800004091A0205090E090D1003101B14040688
:103190001F1E1C1D1C190F1E0510050B140E0217F7
:1031A0000E12120B160114141A12001C1008150727
:1031B000180C140F090507011113011C110C1C0830
:1031C0000414101E021202041D1F0906160209151E
:1031D0000D05180E161F021917070C14040E05030F
:1031E000090B091407161B0813160B1F100A191ECA
:1031F00007031C051414FFFFFFFFFFFFFFFFFFFF86
:10320000FFFFFFFFFFFFFFFFFFFFFFFFFFFFFFFFCE
:10321000FFFFFFFFFFFFFFFFFFFFFFFFFFFFFFFFBE
:10322000FFFFFFFFFFFFFFFFFFFFFFFFFFFFFFFFAE
:10323000FFFFFFFFFFFFFFFFFFFFFFFFFFFFFFFF9E
:107C00000C942A3E0C94473E0C94473E0C94473EFD
:107C10000C94473E0C94473E0C94473E0C94473ED0
:107C20000C94473E0C94473E0C94473E0C94473EC0
:107C30000C94473E0C94473E0C94473E0C94473EB0
:107C40000C94473E0C94473E0C94473E0C94473EA0
:107C50000C94473E11241FBECFE5D8E0DEBFCDBF58
:107C600010E0A0E6B0E0ECE8FEE702C005900D925F
:107C7000A236B107D9F710E0A2E6B0E001C01D922C
:107C8000A038B107E1F70E94213F0C94453F0C94C6
:107C9000003E0C94000008955F9BFECF8CB1E6E699
:107CA000F0E05F9BFECF8CB1819380E0E038F80775
:107CB000C1F75F9BFECF8CB10895CF93DF936091A6
:107CC000600070916100A0916200B0916300C6E60F
:107CD000D0E0A038B105A1F483E0FB018093570008
:107CE000E89507B600FCFDCF85E0FB0180935700C7
:107CF000E89507B600FCFDCF60587F4FA0E0B0E0EC
:107D0000588141E09D01260F371F898190E0982F0F
:107D10008827850F911D0C01F90140935700E895C4
:107D200011241296229680E0C038D80791F67093FD
:107D3000610060936000B0936300A0936200DF91E4
:107D4000CF91089525E08091600090916100FC0141
:107D500020935700E89507B600FCFDCF089523E077
:107D60008091600090916100FC0120935700E8959C
:107D700007B600FCFDCF08955F9BFECF2CB15F9B43
:107D8000FECF8CB190E0982F8827820F911D9093A1
:107D900065008093640041E020E833E10C01F901C3
:107DA00040935700E895112483E0F9018093570030
:107DB000E89507B600FCFDCF25E080E893E1FC01E3
:107DC00020935700E89507B600FCFDCF0895CF93A8
:107DD000DF930E94BC3EC0E0D0E00DC088B394E0C9
:107DE000892788BB0E944C3E0E945D3E5D9BFECF72
:107DF0008EE78CB921968091640090916500C81738
:107E0000D90760F3209160003091610083E0F901AF
:107E100080935700E89507B600FCFDCF85E0F90197
:107E200080935700E89507B600FCFDCF81E1809371
:107E30005700E8955D9BFECF83E48CB9DF91CF912D
:107E400008950E943A3F84E087BBC2985F9BFECFB3
:107E50008CB1823519F40C940000F7CF8A3219F4F2
:107E60000E94E73EF2CF843581F75D9BFECF84E52B
:107E70008CB9EBCF10BC8BE089B988E18AB986E870
:107E800080BD8CB15F99FDCF0895FFCF0014FFFF37
:107E9000FFFFFFFFFFFFFFFFFFFFFFFFFFFFFFFFF2
:107EA000FFFFFFFFFFFFFFFFFFFFFFFFFFFFFFFFE2
:107EB000FFFFFFFFFFFFFFFFFFFFFFFFFFFFFFFFD2
:107EC000FFFFFFFFFFFFFFFFFFFFFFFFFFFFFFFFC2
:107ED000FFFFFFFFFFFFFFFFFFFFFFFFFFFFFFFFB2
:107EE000FFFFFFFFFFFFFFFFFFFFFFFFFFFFFFFFA2
:107EF000FFFFFFFFFFFFFFFFFFFFFFFFFFFFFFFF92
:107F0000FFFFFFFFFFFFFFFFFFFFFFFFFFFFFFFF81
:107F1000FFFFFFFFFFFFFFFFFFFFFFFFFFFFFFFF71
:107F2000FFFFFFFFFFFFFFFFFFFFFFFFFFFFFFFF61
:107F3000FFFFFFFFFFFFFFFFFFFFFFFFFFFFFFFF51
:107F4000FFFFFFFFFFFFFFFFFFFFFFFFFFFFFFFF41
:107F5000FFFFFFFFFFFFFFFFFFFFFFFFFFFFFFFF31
:107F6000FFFFFFFFFFFFFFFFFFFFFFFFFFFFFFFF21
:107F7000FFFFFFFFFFFFFFFFFFFFFFFFFFFFFFFF11
:107F8000FFFFFFFFFFFFFFFFFFFFFFFFFFFFFFFF01
:107F9000FFFFFFFFFFFFFFFFFFFFFFFFFFFFFFFFF1
:107FA000FFFFFFFFFFFFFFFFFFFFFFFFFFFFFFFFE1
:107FB000FFFFFFFFFFFFFFFFFFFFFFFFFFFFFFFFD1
:107FC000FFFFFFFFFFFFFFFFFFFFFFFFFFFFFFFFC1
:107FD000FFFFFFFFFFFFFFFFFFFFFFFFFFFFFFFFB1
:107FE000FFFFFFFFFFFFFFFFFFFFFFFFFFFFFFFFA1
:107FF000FFFFFFFFFFFFFFFFFFFFFFFFFFFFFFFF91
:00000001FF
